:020000040000FA
:100000006C2800000000000009001108820760341D
:100010003134323433346134343435343634623448
:1000200037343834393463342A3430342334643444
:100030001530840089018316081483120808800093
:10004000840A890A19300402031D1B280800153090
:1000500084008901000888008316081208155530AD
:100060008900AA30890088148312000000008316DA
:10007000081E34288312840A890A19300402031DD9
:100080002A2808008D0050308E008E0B45288D0BDD
:100090004328080090008615033042208611033063
:1000A0004220900B4B280800910104309200FE3052
:1000B0006500A0304220060E940004309300910A9F
:1000C000940C031C0528930B5F2803148316850DDD
:1000D0008312920B592800348501030165008601C3
:1000E000F0306600831681138312F0304A20182006
:1000F0008F010F0886009B201530DA20031D792818
:100100002A30110203198E2804300F068F00860052
:100110007928C83042208F0B8928792802300F04B3
:1001200086009B201530EE209B201530DA20031D21
:100130007528272079289901030165000608F03900
:10014000F03A031D9C28F0304220060808308B004E
:1001500063005420FF39910003199C28F03042209D
:1001600004301902031DC728D320031DBB284030CB
:100170004A20110808001B30840000088403800016
:10018000840A840A1E300402031DBD289903D3206B
:1001900003199B2840304A201A301907840011089F
:1001A0008000990A9C2823301102031908002A3084
:1001B000110208009E0099011A30190784000008F6
:1001C0009F001E081907840000081F02031D080075
:1001D000990A04301902031DDC2808009E009901C9
:1001E0001A301907840000089F001E0819078400B0
:1001F0001F088000990A04301902031DF028080026
:02400E00F23F7F
:0C4200003100320033003400350036007D
:00000001FF
